:100000000DC025C069C023C022C021C020C01FC0B0
:1000100096C01DC000010517418BFF0011241FBEB3
:10002000CFE9CDBF10E0A0E6B0E0ECECF3E002C019
:1000300005900D92A636B107D9F710E0A6E6B0E01C
:1000400001C01D92AF36B107E1F782D1BDC1D8CF53
:1000500026EB33E003C0F9013197F1F70197D8F7A8
:10006000089596B393FB992790F981E098278091A2
:100070006900880F892B809369008F7090E0089544
:1000800080916700811115C0909168008091640093
:10009000890F809368008091680018161CF086E034
:1000A0008093680080916800873018F082E0809328
:1000B000680008958091680018162CF480916800FB
:1000C00081508093680008958BB780628BBF08953C
:1000D0008BB78F7D8BBF08951895F894A89581B53F
:1000E000886181BD80E481BD78940895F894A895D5
:1000F00084B7877F84BF81B5886181BD11BC789446
:10010000089581E687B9A29A86EC86B90895379852
:100110000895ECDF1092660003C080E190E098DF64
:10012000A0DF892BD1F7D0DF82E087BB85B7806263
:1001300085BF889585B78F7D85BFCADFCECF1F92DB
:100140000F920FB60F9211242F933F934F935F930B
:100150006F937F938F939F93AF93BF93EF93FF938F
:1001600080916800811104C010926A0010926B00A7
:1001700078DF892BD1F110926A0010926D001092F5
:100180006C0010926E00809166008F3F19F08F5FB7
:100190008093660080916600863161F48FEF8093D2
:1001A0006B0080916800811103C086E38093660034
:1001B00067DFBDC08C3B91F48091670091E0892797
:1001C0008093670080916700882319F0109268007F
:1001D000AEC08091650080936800A9C0853309F0A6
:1001E000A6C085E180936600A2C080916700882345
:1001F00019F010926A0099C080916800882371F00C
:1002000080916A008F3F19F08F5F80936A00809120
:100210006B008F3F19F08F5F80936B0080916600B9
:10022000982F9150943108F58091680081110AC08F
:1002300080916500809368008FEF80936A00109230
:100240006B0073C080916B00853140F48091680031
:10025000863020F486E08093680067C08091680053
:10026000809365001092680060C081115EC080912B
:100270006800863069F480916C0090916D00019661
:1002800090936D0080936C008134910508F012DF2B
:10029000349B43C0409161004093600080916200B4
:1002A00080936100309163003093620025B1209308
:1002B000630090E0840F911D830F911D820F911DAB
:1002C000959587959595879520916800213019F42B
:1002D00021E730E002C02BE730E08217930730F4CB
:1002E00080916E008F5F80936E0013C010926E003D
:1002F0008B39910528F083E087BBC09AC4980DC064
:100300008C38910530F083E187BB88B3816188BB6D
:1003100004C082E187BBC49AC09880916E008C3B78
:1003200018F0C8DE10926E00369A10926600FF91A7
:10033000EF91BF91AF919F918F917F916F915F915D
:100340004F913F912F910F900FBE0F901F901895D6
:1003500017BA88E088BB85BB82E087BB83E28FBD8C
:1003600081E083BFCEDE479A8FEF89BD83E090E0C6
:100370006FDE19BC81E090E06BDE85B7877E80611F
:1003800085BFC7DEC0E020916800332727FD309588
:100390008C2F90E028173907B1F3E0916800FF2710
:1003A000E7FDF095EC5EFF4FE491E9BDC091680078
:1003B00081E090E04DDE809168008111E4CF81E022
:0C03C00090E046DEA6DEDFCFF894FFCF11
:0603CC00A9A9A9A9010284
